:030000000219FDE5
:03000B000200AA46
:03002B0002015C73
:03005B000202EBB3
:030073000202D8AE
:1000800002030406080C10182030406080040608A3
:100090000C10182030406080A0C00003070F1F0D17
:1000A0000D0403060D0503030202C2AFC0D0C0E079
:1000B000206214E5256009E473E525F4F58AD2622F
:1000C000D0E0D0D0D2AF3285268AC262E526F46075
:1000D0002F30682520720DD0E0D0D0C292C290C2DD
:1000E00091D2AF32C292C290C291206F0C206609A9
:1000F000740AD5E0FDE57B4290D0E0D0D0D2AF329B
:10010000758A00C28DD26201F901B9306805206696
:1001100002D29201B9306805206602D29101B9304D
:100120006805206602D29001B9C29530680A20663F
:10013000077408D5E0FDD29201B9C29430680A2054
:1001400066077408D5E0FDD29101B9C29330680A00
:100150002066077408D5E0FDD29001B9C2AFC2ADE8
:1001600053E6EFC0D0C0E0D2D3D2AFC2CEE52A6012
:1001700007207449152A21BD7800790020742EE5E6
:1001800080307E01F430E70278FF53DACF207E031F
:1001900043DA20307E0343DA10C2D8C271E58030E2
:1001A0007E01F430E70279FFC3E89970CB30610338
:1001B000752A40207403752A40885CD27020740D23
:1001C000E52B6004152B21CD43DA01C2D820700243
:1001D00021E0A85C206102C27020740221DE882226
:1001E0007882B60403852224C3E52594404002D2D8
:1001F0006420CF0AD0E0D0D043E610D2AD32C2CFD7
:10020000053A7802E52A6005307402152AC3E55CD8
:1002100094014005755F00412A756000756900E52D
:100220005F2401F55F5003755FFF7982B7020D30DF
:100230006E1DC3E52294324016854C227982B703A5
:100240000E306E0BC3E52294324004798E8722C3B0
:10025000E5239522600840041523415E0523D8CA92
:100260000569E56970021569D56A63756A017805E3
:10027000C3E569956B4057C3E569956C50087801F3
:10028000756A03020292C3E569956D5005780175A0
:100290006A01C3E5629524401E7982B7040241C316
:1002A000206E14852462E569046003856B69756AB4
:1002B0000175233C0202CEE5622850057562FF41BC
:1002C000C3F562E5620470067560FF7569FFD0E0F2
:1002D000D0D043E610D2AD32C2AF53E67F7592FA6A
:1002E0007593FFC260759104D2AF32C2AF53E6EF8F
:1002F000C2ADC0D0C0E0C0F0D2D3D2AFA8FBA9FC41
:10030000C2D8307102615253DACF207E0343DA1033
:10031000307E0343DA20D271E580307E01F420E79D
:1003200002612988278928A13753DACF207E034329
:10033000DA20307E0343DA10C2D8C271307402A1D1
:10034000237800E580307E01F430E702A123885C49
:10035000A10B53DACF207E0343DA20307E0343DA49
:1003600010C271206102812B53DACF207E0343DA61
:1003700010307E0343DA20C2D8D27188578958C31F
:10038000E89555F8E99556F97B007E087A00C3E8B0
:10039000948CE994005005755B00811D882178A23A
:1003A000E6A8216055C3E894C8E994005008E4D257
:1003B000E4FB7A0A61F8C3E89468E994015008E420
:1003C000D2E3FB7A0F61F8C3E894D0E994025008B5
:1003D000E4D2E2FB7A1E61F8C3E894A0E9940550E8
:1003E00008E4D2E1FB7A3C61F8C3E89498E9940808
:1003F0005008E4D2E0FB7A787E00C3E89559FCE926
:10040000955AFD30E70AECF42401FCEDF43400FDCC
:10041000755B00C3EC9AED9E5003755B01885989AA
:100420005A8557558558567802A10BC3E89527F889
:10043000E99528F9307C0281EF307B0281EF307A38
:100440000281E8207502814EE9FDE8FC816DE9C377
:1004500013F9E813F830790281E8E9C313F9E813D6
:10046000F830780281E8E9C313FDE813FC20612C21
:0F047000C3EC941CED940240028184ED701EC316
:10047F00EC94C850180529E52970021529C3E52900
:10048F00940A5002A123755C00D270A123E5296064
:10049F000215297400207F037896E624FAFEE434CF
:1004AF0000FFC3EC9EFCED9FFD50067800790081A4
:1004BF00EFC3EC94FFED9400400678FF790081EFD5
:1004CF00EC8572F0A4C5F0A2F733F879004003026F
:1004DF00050B78FF790002050BE9C313F9E813F850
:1004EF00307C0EE9600278FFC3E81338F8E434007B
:1004FF00F9C3E894FFE99400400278FF885CD2705A
:10050F00206102A123741FF4552F4BF52FC274EBFA
:10051F007002D274752A40307403752A0A30610252
:10052F00A13720740353DAFE207403752B20D0F00B
:10053F00D0E0D0D0D2AD43E6103279010205677911
:10054F0003020567790A020567791E020567796458
:10055F0002056779C80205677817E4D5E0FDD8FA78
:10056F00D9F6227A147B7802058E7A107B8C0205DD
:10057F008E7A0D7BB402058E7A0B7BC802058E79BD
:10058F0002E4C294D5E0FDD291D5E0FDC291D5E051
:10059F00FDD294D5E0FDE920E002D29230E002D204
:1005AF0090E573D5E0FDE920E002C29230E002C28F
:1005BF00907496D5E0FDD9C9EAF8D5E0FDD8FBDBFC
:1005CF00BEC29422C37C007D0075F00005F0EA33B3
:1005DF00FAEB33FB50F6EB13FBEA13FAC3E9FFE830
:1005EF00FEE89AF8E99BF95004EFF9EEF8B3EC3313
:1005FF00FCED33FDD5F0DFEDF9ECF822E889F08A58
:10060F0020D2D4F8A9F07B0030F70B7BFFF4240144
:10061F00F8E9F43400F9E88520F0A4ADF0F8E985A5
:10062F0020F0A4AFF0FEED2EF974003FFA7C04C366
:10063F00EA13FAE913F9E813F8DCF48BF030F70A50
:10064F00E8F42401F8E9F43400F9E889F0C2D4F8A9
:10065F00A9F0227882B60403020701C3E55C94195E
:10066F00401EE52D54067018206E3678057994E7F4
:10067F00146007780A1460027812C3E54198401F8E
:10068F00306E098564627569FF756A01852224E4FD
:10069F00F544F545F546F547F548C26E020701D218
:1006AF006E7994E7147013E523F43333F913F8E9F3
:1006BF00540104F9E854FE0206F5E714147014E52A
:1006CF0023F4333333F913F8E9540304F9E854FCF2
:1006DF000206FDE523F433333333F913F8E95407F6
:1006EF000404F9E854F8C39440F8E99400F98844F5
:1006FF00894522C3E54113F9E54013F8C3E5449852
:10070F00F8E54599F9500CC3E89480E994FF401639
:10071F00020739C3E8947FE9940050030207397840
:10072F007F7900020739788079FF8849894A22E565
:10073F00492546F8E54A3547F9854A20E43007014F
:10074F00F43548FA30E709C3EA94F0401502077709
:10075F00C3EA940F500302077778FF79FF7A0F02ED
:10076F000777780079007AF0C3E5249561500AC3C2
:10077F0074019524500B020795E54A20E70E0207F6
:10078F0095E54A30E706884689478A482278A5E6E4
:10079F00FAC3E54933F8E54A33F9D10BE930E70BF2
:1007AF00C3E89480E994FF4013E1CFC3E8947FE955
:1007BF0094005002E1CF787F7900E1CF788079FF04
:1007CF00E820E715C3E52398F84009C3E8940140F2
:1007DF00030207F678010207F6E8F424012523F84F
:1007EF0040030207F678FF884B2278A6E6FAA8475F
:1007FF00A94812060BE930E70CC3E89401E994FF0E
:10080F00401602082BC3E894FFE994005003020836
:10081F002B78FF790002082B780179FFE920E71583
:10082F00C3E54B98F84009C3E8940140030208520E
:10083F007801020852E8F42401254BF8400302081E
:10084F005278FF88242278FFC26420693D206A1203
:10085F00D264C3E541940A4009C3E5259440500290
:0D086F00C26479A1E76023E541601F74FFBA
:10087C008541F0848539F0306A0375F005A4F8C51C
:10088C00F0600278FFC3E895645002A86488632284
:10089C00C3E5409440E5419401E56350031401AD78
:1008AC00046002F563227883E6F520120F2A75E8BE
:1008BC009012054975E890E5E820ECFBA8BDA9BEAF
:1008CC00120FD0756E2C756F00C3740013FD742C51
:1008DC00606613FC742C2CFC74003DFDECFAEDFBF3
:1008EC00C3E89AE99B4014E56E242CF56EE56F3451
:1008FC0000F56FEA2CFAEB3DFB80E5AE6EAF6FC3F3
:10090C00E56F13F9E56E13F8C3E913F9E813F87AF8
:10091C0003C3E913F9E813F8DAF7AA201A7009757A
:10092C006E00756F000209441AEA6008EE28FEEFAB
:10093C0039FFDAF88E6E8F6F2275E890227883E695
:10094C00FFE5E820ECF7A8BDA9BE0570C3E57094DF
:10095C00084052757000E9FA79A0E76044EA700724
:10096C00E571601B02097FC3E895716010E5715059
:10097C0006600C1402098B0460F902098BE571F511
:10098C0071C3946D401B7561C0C3940440137561B1
:10099C0080C39404400B756140C39404400375619B
:1009AC000075BB0622EFC39401601F742C601BC33F
:1009BC00E894FFE994035012C3E8956EE9956F50E3
:1009CC0009E561600C15610209DDE561F460020561
:1009DC0061A861C3E524985002A824C3E89562403D
:1009EC000AA862E562F4600385626188258826E5C1
:1009FC0070B4070375BB1022743279A787F0A4C5B5
:100A0C00F0A2F733F8C3E895614002A86188228808
:100A1C0024882588268864227540007541F022C2FE
:100A2C00AF75C820A8CCA9CDAA3A30CF010A75C899
:100A3C0024D2AFAB3BAC3C883B893CC3E89BF8E988
:100A4C009C206908F930670261374194AD3D8A3DBD
:100A5C00F9EA9DFA600478FF79FFAE3EAF3F8B3E1A
:100A6C008C3FA83BA93CC3E89EF8E99FF9C3E5413C
:100A7C0013FBE54013FAE82AF540E93BF541500633
:100A8C007540FF7541FF41DEAA40AB41AC40AD4122
:100A9C007E047F02C3EB940440021E1FC3EB940838
:100AAC0040021E1FC3ED13FDEC13FCDEF7C3EA9CE2
:100ABC00FAEB9DFBEF6009C3E913F9E813F8DFF7D4
:100ACC00EA28FAEB39FB8A408B4150067BFF8B40BE
:100ADC008B41C3EB94025002D2673069047F0361EF
:100AEC00097892E6FFC3E537948240110FC3E537CE
:100AFC0094A040010FC3EF940640027F057E02E5EF
:100B0C0041C4540FF9E541C454F0F8E540C4540F06
:100B1C0028F8C3E89EFAE99400FB4009C3EA940262
:100B2C00EB940050047A02E4FB6183AA40AB41EBE6
:100B3C00C4FEEAC4540F4EFCC3EA9CFAEB9400FBCF
:100B4C00C3E813C313F8EA28FAEB3400FB8A408B92
:100B5C0041C3EB94024002C2677802EBC4FE7B00F7
:100B6C00EAC4540F4EFAC3EA98FA4005C3940250F3
:100B7C00027A027892E6FF30600261838551928599
:100B8C005293D26043E680C3E49AF8E49BF9306751
:100B9C0002810FE8FAE9FBD3E913FDE813FC885155
:100BAC008952C3EF94036038EF20E00DE82CF8E98C
:100BBC003DF9ECFAEDFB020BD8E828F8E939F9C35A
:100BCC00E82402F8E93400F97AFE7BFFC3EF9403C2
:100BDC00400E8A538B54884D894E8C4F8D508143D7
:100BEC00885389548A4D8B4E8C4F8D5030691275B9
:100BFC0053F07554FF754FF07550FF7551F07552E9
:100C0C00FF8143E8FAD3E813FC8851C3EF940360E7
:100C1C0020EF20E007E82CF8ECFA812FE8282402DA
:100C2C00F87AFEC3EF940340088A53884D8C4F81A9
:100C3C004388538A4D8C4FE568C3335002646BF57F
:100C4C0068306002814D753402D26043E680E52D38
:100C5C0054066034A840A941C3E913F9E813F8C35A
:0F0C6C00E913F9E813F8306904E92440F9C2AF3D
:100C7B0053E67F759100C3E498F594E499F5957567
:100C8B009104D26043E680D2AF22D26575430075E2
:100C9B002000306C03752040020CB4D26575430004
:100CAB00752040306C037520007801790120672096
:100CBB00E52D54066002C2657914E541C31370013A
:100CCB0004F8C3941440027814306904781B791B20
:100CDB00206010E543600C306903D53404D26DA15C
:100CEB005791550543E59BF45440B52002A1413083
:100CFB00690908C3E89940011881DB20650A08C31C
:100D0B00E899400281B481DBC265C2AF53E67F75BF
:100D1B0091003067127594007595FE759104D26041
:100D2B0043E680D2AF81B4AE40AF41C3E49EF594AD
:100D3B00E49FF595A126C3E5339401500281B430AD
:100D4B00650281B4D802A15581DBC26DC2AF53E6F7
:100D5B007F759100855394855495759104854D92BB
:100D6B00854E93D26043E680D2AFE52D54066008E2
:100D7B00206A020533020D93306D0D206C0A20653D
:100D8B00071581158102160822780030640530653D
:100D9B00027801E53775F007A4F9E5F028F5F0E9DD
:100DAB00A2F013A2F113A2F213F537C394785003F8
:100DBB00753778C3E53795384008D266C292C29032
:100DCB00C291306002A1CD854F92855093D2604382
:100DDB00E68022207D16C2AF754202C294D29530B6
:100DEB006202D290D2AF759F11020FCDC2AF754286
:100DFB0002C294D293306202D292D2AF759F11028B
:100E0B000FCD307243207D20C2AF75420390013A63
:100E1B00757B10C290C293306204D291C12BD294D5
:100E2B00D2AF759F01020FCDC2AF75420390013A4D
:100E3B00757B10C292C295306204D291C14BD29491
:100E4B00D2AF759F21020FCD207D17C2AF75420324
:100E5B00900115C290306202D291D2AF759F010200
:100E6B000FCDC2AF754203900115C292306202D210
:100E7B0091D2AF759F21020FCD207D16C2AF754267
:100E8B0004C295D293306202D291D2AF759F2102E8
:100E9B000FCDC2AF754204C293D295306202D2918C
:100EAB00D2AF759F01020FCD307243207D20C2AFB0
:100EBB00754205900129757B20C291C29430620462
:100ECB00D292C1D1D295D2AF759F11020FCDC2AFC5
:100EDB0075420590014B757B08C291C29430620438
:100EEB00D290C1F1D293D2AF759F11020FCD207D5D
:100EFB0017C2AF75420590010BC291306202D292BC
:100F0B00D2AF759F11020FCDC2AF75420590011F75
:100F1B00C2913062EBD290D2AF759F11020FCD20F0
:100F2B007D16C2AF754206C293D294306202D29242
:100F3B00D2AF759F01020FCDC2AF754206C295D2DB
:100F4B0094306202D290D2AF759F21020FCD3072D6
:100F5B0043207D20C2AF75420190014B757B08C2C7
:100F6B0092C295306204D290E177D293D2AF759F43
:100F7B0021020FCDC2AF754201900129757B20C2B2
:100F8B0090C293306204D292E197D295D2AF759F03
:100F9B0001020FCD207D17C2AF75420190011FC218
:100FAB0092306202D290D2AF759F21020FCDC2AFA9
:100FBB0075420190010BC290306202D292D2AF7592
:100FCB009F01C26622900109757B00C292C290C23A
:100FDB0091C295C293C294C262227880760708763A
:100FEB00070876010876040876FF0876FF0876096D
:100FFB00087602087601087601788C76010876006F
:10100B000876B40876FF0876FF0876FF08760308A3
:10101B0076FF0876010876FF0876250876D00876E5
:10102B00780876C80876040876FF087601087600FB
:10103B0008767A08760A08760108760108760008A1
:10104B0076FF087600227887E6FFC272BF0302D2D2
:10105B00727888C27DE630E102D27DC27E7889E665
:0E106B0030E102D27EC3EF94026008758E0160
:10107900D273021083758E00C273227880E61490B1
:1010890000809378A5F67881E6149000809378A67D
:10109900F67886E61490008D9378A7F6789FE6F89F
:1010A900700108C3E8941140027811E82828F56B0B
:1010B900256B256B28F56C256B2828F56D7886E658
:1010C900F539C394025003753902789CE67538FFE7
:1010D900B402037538A0B4030375388278A3E61403
:1010E90090009A93F566120FD022227896E6FA7844
:1010F90097E6FB7888E6B40305C3EB940EFB307FD3
:10110900047A007BFFC3EB9AFCC3948250027C8271
:101119007572000572EC8572F0A4C3E5F0947D4008
:10112900F222D27F11F41205587A007B007C10124A
:10113900054EE55C2AFA74003BFBDCF37C04C3EB47
:1011490013FBEA13FADCF7FEC27F11F422E5EF2064
:10115900E6037520000520903FFFE5201460069006
:101169001DFF1460009304600375EF1253D9BF7516
:1011790081C043FF8012054975EF0243B203E5B30D
:10118900240220E70DF521E5E320E0068521B3439C
:10119900E301120FD07580FF75A40075F19175D424
:1011A9007F75900075A53F75F23F75D50075A6014D
:1011B90075E241120FD0E4F8F6D8FD756801120FF7
:1011C900E512165F78988673753001C2AF12056211
:1011D9001205721205581205791205581205801266
:1011E900055812178212056212056212055DC2AF17
:1011F90078FA79FA308707D9FBD8F7021C00115120
:10120900118411F311F478988673120FD075881030
:1012190075890275C82475910475D84075A8227519
:10122900B80275E690759B80759D0075D10E75BCE9
:101239005875BB0675BA1175E880120549D2AF1207
:1012490008B275360053DACF207E0343DA20307EA8
:101259000343DA1043DA01C2D8C271120562D261BE
:101269007B037A0CE55B70077A0CDB030211F7123A
:1012790005582070030211F7C270E55CC39402405F
:10128900E1E52F541F855E5DF55EB55DD5DAD5C202
:101299006153DACF207E0343DA20307E0343DA102C
:1012A900C2D8C27178A2E67008D274E52F54E0F56D
:1012B9002FC27575290012055D307409C3E529949B
:1012C9000A4002D27512054E78023074027800C3C2
:1012D900E55C9840F0C2AF120572120572120572F0
:1012E900D2AF120562754C0012054E788CE6C39494
:1012F9000150030213C7E530C3940150030213C719
:10130900207435C3E55C94FF50030213C7C2AF12C2
:101319000587D2AF12055DC3E55C940150EFC2AFFA
:10132900120572120553120572D2AF12055DC3E59B
:101339005C94FF40E90218077F05D27F11F412057A
:101349005DC2AFC27F11F4AE5CC3E55C947FD2AFDE
:101359004076120549C2AF120587D2AFDFDC312BC7
:10136900C3EE94057897F61205621216A112178A30
:101379007F0AD27F11F412055DC2AFC27F11F4AEAC
:101389005CC3E55C947FD2AF50E6120549C2AF1247
:101399000572120553120572D2AFDFD6312BEE2436
:1013A900037896F61205621216A11217B912055D95
:1013B90011F4C3E55C94FF50026109021807C3E503
:1013C9005C954C4003855C4C12055D78017988E792
:1013D900B403027805C3E55C98400241F1C2AF123B
:1013E9000587120587120587D2AF1205627530008D
:1013F900E4F531F5320531E531F4703F0532789A7B
:10140900E67819146012783214600D787D1460083A
:1014190078FA146003753200C3E53298401D120F43
:10142900D0120549153275310078998673C2AF1209
:101439000587D2AF7898867312055D120553E52AA0
:10144900700530740221F778012074027806C3E52B
:101459005C9840A112055DE52A70030211F7C2AF3D
:0E146900120FD0E4F522F523F524F525F52623
:10147700F567D2AF7885E6C333F565E4F544F545FE
:10148700F546F547F548F570F52CF52DF5377570E8
:101497000875BB10120549120945E5E820ECFBA8C1
:1014A700BDA9BEE97001F888711209497570087500
:1014B700BB101151C2AF7561FF120A048522618505
:1014C7002262852263D2AF75220175240175250139
:1014D700752601856069756A017888E6B40307C2D5
:1014E7007D307602D27DD268D269753300120F2A19
:1014F700120F59120A24120A2B120A24120A2B124B
:101507000A24120CA6120662120D94120DDE120A9C
:101517002B120C95306E0312070220670312085531
:1015270030670312089C120D94120E0D120A2B122B
:101537000CA6306E0312073E120D94120E84120A87
:101547002B120C95306E0312079C120D94120EB3DA
:10155700120A2B120CA6306E031207F9120D941201
:101567000F2A120A2B120945120C95120D94120F0D
:1015770059120949120A2B30692C85646185646206
:10158700856069756A0179187A0CC3E53399400952
:10159700C269D26A8A350215ADC3E55C940140037E
:1015A700021509021610306A1D206C1AE5351470F1
:1015B70006C26AD26BA109F535C3E55C9401400305
:1015C700021509021610753600C3E55F940140093C
:1015D700856462856069756A0178FA79A4E76002B3
:1015E7007803C3E55F985021307404E52A601A78C0
:1015F700F0306C058564617820C3E541985002A1FD
:10160700090536E55C6002C113753600C2AF120FDB
:10161700D07887E6FE760211517887EEF6E4F52258
:10162700F523F524F525F526F565752C00752D00B0
:10163700D2AF12055D120FD078A4E66006D292D21F
:1016470091D290307406E52A700221F7788DE6C3AF
:101657009401400241CE61F9901A0D78201216E3E9
:10166700E520B4A50CA31216E3E520B45A0302162D
:1016770081120FE51216A10216A0901A0378807B3B
:101687000A1216E3A308DBF9901A0F788C7B19125C
:1016970016E3A308DBF9901A2822C2AF1217221209
:1016A70016FC901A00740E1216E8A374061216E8B8
:1016B700A374151216E8901A0378807B0A1216E7AE
:1016C700A308DBF9901A0F788C7B191216E7A30889
:1016D700DBF9121735121713901A2822E493F62212
:1016E700E6438F01538FFD75EF0275B7A575B7F107
:1016F700F0538FFE22438F02438F0175EF0275B7B8
:10170700A575B7F1901A0DF0538FFC22901A0D743E
:10171700A5D1E8901A0E745AD1E8227A3079D07898
:1017270020901A40D1E3E520F709A3DAF7227A30AF
:1017370079D0901A40E7D1E809A3DAF922AB74A867
:1017470075BB01027980BB02027981BB03027982F2
:10175700BB04027994BB05027983BB06027986BB79
:1017670007027992BB08027987BB0902799CBB0AF9
:10177700027988BB0B027989E8F7227C051205629A
:10178700DCFB22C2AF120572120579120580120521
:101797008712055312057212057912058012058703
:1017A700120553120572120579120580120587D2A8
:1017B700AF22C2AF12058712058012057912057292
:1017C7001205531205871205801205791205721248
:1017D7000553120587120580120579120572D2AFDB
:1017E70022AE74AF75C2AF1205721205721205727E
:1017F700120553DEF2120587120553DFF8D2AF2226
:1018070012178A121782121782757401757501757E
:1018170076001217E87C05AD5C120562C3ED955C96
:1018270070F5C3E55C9401400AC3E55C94FF40375B
:1018370002184B1217441216A112178AC2AF75EF7E
:1018470012121782DCD10576C3E576940350028025
:10185700C11217820575E5741490009F93F808C3A9
:0F186700E57598500280A8121782121782057437
:10187600C3E574940C50028094120FE51216A1C2AF
:07188600AF75EF121217828B
:0319FD000211567E
:101A00000E061507070104FFFF09020101A55A018F
:101A100000B4FFFFFF03FF01FF25D078C804FF01DA
:091A200000FF0A010100FF00FFB4
:101A40002358503335415357232020202020202075
:101A500023424C48454C4923463333302320202031
:101A60002020202020202020202020202020202076
:101C0000C2AFC2D353D9BF7581C043B20343FF8073
:101C1000752438752503B1C975EF0275E24043F1AB
:101C20008053A47F75D4FFD2877DFA780379E67C50
:101C300010752200752300901DD67B0675249875BB
:101C400025013087028142208708D8FBD9F9DCF7CB
:101C500081B4308708D8FBD9F9DCF781B4B189E4C5
:101C600093A3C39A6004DDC381B4DBDBB17B600264
:101C7000812B7B08E493FAA3B15CDBF87A30B15C8A
:101C8000752200752300B17BEAFCEBFDC3ED94FEE9
:101C9000400EB17B8A278B28ED30E0048A828B834B
:101CA000B17B7AC270D8C3ED94FE601350CEBD00F4
:101CB00025EC60097520007521FF0200008100A855
:101CC00027A9280809D804D90281D3B17FEA89AAB3
:101CD000F281C50D81A0C3ED94035049EDA2E092BD
:101CE000007AC5C3E5829400E583941C50902000DF
:101CF00010438F02438F0175B7A575B7F1F030001F
:101D00001FA827A9280809438F01538FFDD804D99C
:101D100002A12089AAE275B7A575B7F1F0A3A10DBC
:101D2000538FFC817C7AC1BD030CE493A3FAB140CC
:101D3000DCF8B138817C817EAA22AB23B15CEBFA5E
:101D4000EA6222752608C3E52313F523E52213F57D
:101D50002250066323A0632201D526EAB1C9B1C986
:101D600075260AEAF4200102D287300102C287B147
:101D7000C9C3134002C201D526EB22B17FEAFB2082
:101D80008702A17F308702A184752608AE24AF2583
:101D9000C3EF13FFEE13FEB1CDB1C9C3EA13308711
:101DA000024480FA30E703632201C3E52313F523DD
:101DB000E52213F52250066323A0632201D526D91C
:101DC000E52265236523F52222AE24AF250E0FDE22
:101DD000FEDFFCD20122424C48656C693437316326
:041DE000F3300601D5
:00000001FF
